:10000000292864000C1E0128990003142428A30148
:10001000A200FF30A207031CA307031C24280330FF
:10002000A100E73015200928A101FC3EA000A1098C
:10003000031C2028FF300000A00703181B28A0077E
:100040006400A10F1A2808008313031383126400AD
:1000500008008316043099006530980083129030B0
:1000600098009817BB015530BC00AA30BD00FF3086
:10007000BE003610B6103611B611053007206400E8
:100080003B08FF3C031D4528361064003B08003C3C
:10009000031D4B283614640036184F28BB03640038
:1000A000361C5328BB0A64003C08FF3C031D59283A
:1000B000B61064003C08003C031D5F28B6146400C1
:1000C000B6186328BC036400B61C6728BC0A640029
:1000D0003D08FF3C031D6D28361164003D08003CBF
:1000E000031D73283615640036197728BD03640094
:1000F000361D7B28BD0A64003E08FF3C031D812895
:10010000B61164003E08003C031D8728B615640044
:10011000B6198B28BE036400B61D8F28BE0A98133B
:1001200006118316061178308312142006158316E3
:100130000611083083121420981700300120243053
:100140001420981306158316061108308312142004
:1001500098173B08012024301420981306158316A5
:10016000061108308312142098173C08012024300F
:1001700014209813061583160611083083121420D4
:1001800098173D0801202430142098130615831673
:10019000061108308312142098173E0801202430DD
:1001A00014209813061583160611083083121420A4
:0801B0009817053007203D28D7
:02400E00543F1D
:00000001FF
